:020000040000FA
:0400000072EF00F0AB
:0800080082EF00F00C6E240EE3
:10001000036EF40E046E4BEC00F0D8B4CA90D8A472
:10002000CA80FC0FD8A0CA92D8B0CA82036A240E34
:10003000046EF40E076E086ACAB027D8CAB225D873
:100040004DEC00F00304CB6E03C005F004C006F0D5
:100050000050096E0A6E003C0A6A62EC00F008501B
:100060000C2E0AD0BE6E0C0EBD6E07BEBD8A07BC3C
:10007000BD889394CA841200BB6E0C0EBA6E07BE84
:10008000BA8A07BCBA889492F5D700D8D8900732BC
:10009000043203321200086A076A100EF36E043449
:1000A000073608360550075C0650085805E305502A
:1000B000075E0650085AD88003360436F32EEFD771
:1000C0000350120005500902F3CF07F0F4CF08F0F7
:1000D00006500902F350082605500A02F35008267C
:1000E00007501200F86A7F0EAF6E240EAC6E900EB1
:1000F000AB6E00017B6A7A6A7E6A7F6A0F0EC16E00
:10010000E2EF00F09EAAA1EF00F0060EAB1412E1A0
:10011000E1CF30F0E2CF31F0322A15EE00F032506C
:10012000E126000EE222AECFE7FF30C0E1FF31C092
:10013000E2FF1100AE50AE50AB98AB881100ADEFAE
:1001400000F0F2A4ADEF00F0F2940F2A81709390CA
:100150000FBE81820FAE8192110011003250335CCC
:10016000D8B4C8EF00F0332AE9CF03F0EACF04F0A7
:1001700005EE00F03350E926000EEA22EF50036E40
:1001800003C0E9FF04C0EAFFD8801200CCEF00F002
:10019000E868036ED8A012001200326A336A9D8AA2
:1001A000F28EF28C12009D9A05EE00F0000EEE6ABF
:1001B000E82EFDD7326A336A9D8A12009EA8FED7C8
:1001C000AD6E1200700E926EE00E936EC00E946EC5
:1001D00093968A969296899692948994929289920D
:1001E0009290899093988A9894948B9494928B92FD
:1001F00094968B962F6AD1DFD6DF170ED56ED76A0D
:10020000D66AF294F28AD58ED9EC04F0A7DF106E8C
:10021000C20E105CD8A019EF01F0FE0E105CD8A041
:1002200016EF01F0A7EF02F019EF01F0126AA7EF45
:1002300002F010AE53EF01F0126A810E105CD8A4E8
:1002400028EF01F010C012F01368146851EF01F0AC
:10025000910E105CD8A433EF01F010C012F01568B5
:10026000166851EF01F0A10E105CD8A43EEF01F02A
:1002700010C012F01768186851EF01F0B10E105C51
:10028000D8A449EF01F010C012F019681A6851EFB4
:1002900001F0C10E105CD8A451EF01F010C012F0B3
:1002A0001B68A7EF02F01252D8A45BEF01F0A7EF92
:1002B00002F0A7EF02F0810E125CD8A4BDEF01F0AE
:1002C0001328D8A468EF01F010C013F0B9EF01F0C3
:1002D00010C014F03A0E135CD8A47AEF01F0006A53
:1002E000420E056E0F0E066E010E90DE94948B94F6
:1002F000B8EF01F03B0E135CD8A483EF01F09492A9
:100300008B92B8EF01F06E0E135CD8A48EEF01F063
:100310002F90279092968996B8EF01F06F0E135C9C
:10032000D8A499EF01F02F92279292948994B8EF74
:1003300001F0700E135CD8A4A4EF01F02F94279461
:1003400092928992B8EF01F0710E135CD8A4AFEFCE
:1003500001F02F96279692908990B8EF01F0720ED7
:10036000135CD8A4B8EF01F02F98279893988A9837
:100370001368A7EF02F0A7EF02F0910E125CD8A469
:1003800070EF02F01528D8A4CAEF01F010C015F0E4
:100390006CEF02F010C016F01652D8A421EF02F054
:1003A0003A0E155CD8A4E0EF01F0006A420E056E2B
:1003B0000F0E066E010E2ADE94948B941EEF02F04F
:1003C0003B0E155CD8A4E9EF01F094928B921EEFDE
:1003D00002F06E0E155CD8A4F4EF01F02F90279078
:1003E000929689961EEF02F06F0E155CD8A4FFEF6F
:1003F00001F02F922792929489941EEF02F0700ED2
:10040000155CD8A40AEF02F02F9427949292899257
:100410001EEF02F0710E155CD8A415EF02F02F96B6
:100420002796929089901EEF02F0720E155CD8A468
:100430001EEF02F02F98279893988A981568A7EFD7
:1004400002F03A0E155CD8A432EF02F016501624D2
:10045000006E420E056E0F0E066E010E06EC00F0E9
:100460006BEF02F03B0E155CD8A43BEF02F09492C8
:100470008B826BEF02F06E0E155CD8A445EF02F094
:100480002F80929689866BEF02F06F0E155CD8A4D0
:100490004FEF02F02F82929489846BEF02F0700E7E
:1004A000155CD8A459EF02F02F84929289826BEFE9
:1004B00002F0710E155CD8A463EF02F02F869290C3
:1004C00089806BEF02F0720E155CD8A46BEF02F01E
:1004D0002F8893988A881568A7EF02F0A7EF02F09B
:1004E000A10E125CD8A485EF02F01728D8A47DEFE6
:1004F00002F010C017F081EF02F010C018F07DEC90
:1005000003F0A7EF02F0A7EF02F0B10E125CD8A43F
:100510009AEF02F01928D8A492EF02F010C019F057
:1005200096EF02F010C01AF0A9EC04F0A7EF02F069
:10053000A7EF02F0C10E125CD8A4A7EF02F01B28AF
:10054000D8A4A7EF02F010C01BF0A3EC04F02752D0
:10055000D8B47AEF03F027A0D4EF02F03EC021F028
:100560003FC022F048C01FF049C020F0D7CF2DF087
:100570000FC02EF022BED2EF02F02252D8A4D4EF48
:1005800002F02150D8A4D4EF02F020502E5CD8A065
:10059000D4EF02F0D8A4D2EF02F01F502D5CD8A007
:1005A000D4EF02F0ECEC04F027A2FDEF02F040C023
:1005B00021F041C022F04AC01FF04BC020F0D7CF3D
:1005C0002DF00FC02EF022BEFBEF02F02252D8A475
:1005D000FDEF02F02150D8A4FDEF02F020502E5C78
:1005E000D8A0FDEF02F0D8A4FBEF02F01F502D5C65
:1005F000D8A0FDEF02F011EC05F027A426EF03F0E0
:1006000042C021F043C022F04CC01FF04DC020F08A
:10061000D7CF2DF00FC02EF022BE24EF03F02252D0
:10062000D8A426EF03F02150D8A426EF03F02050E1
:100630002E5CD8A026EF03F0D8A424EF03F01F50BF
:100640002D5CD8A026EF03F036EC05F027A64FEF7F
:1006500003F044C021F045C022F04EC01FF04FC04F
:1006600020F0D7CF2DF00FC02EF022BE4DEF03F0BB
:100670002252D8A44FEF03F02150D8A44FEF03F03B
:1006800020502E5CD8A04FEF03F0D8A44DEF03F01C
:100690001F502D5CD8A04FEF03F05BEC05F027A8AE
:1006A00078EF03F046C021F047C022F050C01FF0A1
:1006B00051C020F0D7CF2DF00FC02EF022BE76EF24
:1006C00003F02252D8A478EF03F02150D8A478EF99
:1006D00003F020502E5CD8A078EF03F0D8A476EF7A
:1006E00003F01F502D5CD8A078EF03F082EC05F0EA
:1006F0007BEF03F00F6A06EF01F06E0E175CD8A4D3
:10070000B7EF03F02FA0B2EF03F02780D7CF2DF083
:100710000FC02EF0185080080D6E000ED8A0FF0FED
:100720000E6ED8900D34016E0E34026E01C034F09E
:1007300002C035F034C001F035C002F001502D2464
:100740001F6E02502E20206E000E216A2122226A86
:1007500021C03EF022C03FF01FC048F020C049F049
:10076000B5EF03F0279092968996A1EF04F06F0EF3
:10077000175CD8A4F1EF03F02FA2ECEF03F027826F
:10078000D7CF2DF00FC02EF0185080080D6E000E40
:10079000D8A0FF0F0E6ED8900D34016E0E34026E8D
:1007A00001C036F002C037F036C001F037C002F0A9
:1007B00001502D241F6E02502E20206E000E216A43
:1007C0002122226A21C040F022C041F01FC04AF01D
:1007D00020C04BF0EFEF03F0279292948994A1EFA1
:1007E00004F0700E175CD8A42BEF04F02FA426EFB2
:1007F00004F02784D7CF2DF00FC02EF018508008BA
:100800000D6E000ED8A0FF0F0E6ED8900D34016E45
:100810000E34026E01C038F002C039F038C001F069
:1008200039C002F001502D241F6E02502E20206E80
:10083000000E216A2122226A21C042F022C043F028
:100840001FC04CF020C04DF029EF04F02794929285
:100850008992A1EF04F0710E175CD8A465EF04F043
:100860002FA660EF04F02786D7CF2DF00FC02EF013
:10087000185080080D6E000ED8A0FF0F0E6ED89095
:100880000D34016E0E34026E01C03AF002C03BF02E
:100890003AC001F03BC002F001502D241F6E0250FF
:1008A0002E20206E000E216A2122226A21C044F0EF
:1008B00022C045F01FC04EF020C04FF063EF04F09F
:1008C000279692908990A1EF04F0720E175CD8A43D
:1008D000A1EF04F02FA89EEF04F02788D7CF2DF0CA
:1008E0000FC02EF0185080080D6E000ED8A0FF0F1C
:1008F0000E6ED8900D34016E0E34026E01C03CF0C5
:1009000002C03DF0216A226A3CC01FF03DC020F0C9
:100910002D501F24236E2E502020246E000E2120E7
:10092000256E000E2220266E25C046F026C047F018
:1009300023C050F024C051F0A1EF04F02798939801
:100940008A98176812001B6812001D6812001C6844
:100950001200420E195CD8A4BEEF04F01A52D8A4BB
:10096000B8EF04F0C7EC04F093968A96BAEF04F05F
:1009700093968A861AC029F0C5EF04F07B0E195CA5
:10098000D8A4C5EF04F0C7EC04F019681200276A78
:100990009296899692948994929289929290899053
:1009A00093988A9894948B9494928B9294968B9625
:1009B000120093968A96929689969294899492922E
:1009C00089929290899093988A9894948B94949217
:1009D0008B9294968B9612002FB0F3EF04F0279031
:1009E0009296899612002780D7CF2DF00FC02EF057
:1009F00034C001F035C002F001502D241F6E0250AA
:100A00002E20206E000E216A2122226A21C03EF093
:100A100022C03FF01FC048F020C049F08076929677
:100A200012002FB218EF05F02792929489941200C9
:100A30002782D7CF2DF00FC02EF036C001F037C07F
:100A400002F001502D241F6E02502E20206E000E49
:100A5000216A2122226A21C040F022C041F01FC039
:100A60004AF020C04BF08074929412002FB43DEFF6
:100A700005F027949292899212002784D7CF2DF007
:100A80000FC02EF038C001F039C002F001502D2403
:100A90001F6E02502E20206E000E216A2122226A33
:100AA00021C042F022C043F01FC04CF020C04DF0E6
:100AB0008072929212002FB664EF05F02796929002
:100AC0008990120081EF05F02786D7CF2DF00FC057
:100AD0002EF03AC001F03BC002F001502D241F6EF1
:100AE00002502E20206E000E216A2122226A21C08F
:100AF00044F022C045F01FC04EF020C04FF080707F
:100B0000929012002FB88AEF05F0279893988A9850
:100B1000ABEF05F02788D7CF2DF00FC02EF0216A5C
:100B2000226A3CC01FF03DC020F02D501F24236ED0
:100B30002E502020246E000E2120256E000E222033
:100B4000266E25C046F026C047F023C050F024C0D2
:0A0B500051F0817893981200FFD74E
:020000040030CA
:0300010006191FBE
:020005008D80EC
:060008000FC00FE00F40E5
:00000001FF
